:1000000002308A00732A0000D3346D38EC32202A83
:10001000E832F236EF36653AE8327210A0060A008E
:10002000533A613B3A10253220147039EF3165376D
:10003000F430A9060A00533A613B781DA0124C32F5
:100040002838F237E3326E3AE1140D050000533AD6
:10005000613B791DA0124C322838F237E3326E3AF8
:10006000E1140D050001533A613B7A1DA0124C3298
:100070002838F237E3326E3AE1140D05000083169A
:100080008611831286110830F80046280000F81700
:100090005728F813BD0C03188615031C8611781712
:1000A00057287813F80B4A285528000086153F304A
:1000B0008400840B59280000F81B4928781B51281C
:1000C0000800831603178C170C140000000083121D
:1000D0000C087F390319A5280313B40003170D0872
:1000E0000313B50003170F080313B6003408BD004F
:1000F0003F20350803178D000313360803178F00C0
:1001000083168C170C140000000083120C0D0E0DCA
:100110007F390319A5280313B40003170D0803132F
:10012000B50003170F080313B6003408BD003F20C5
:10013000350803178D000313360803178F008D0A47
:1001400003198F0A03136128031703138A110A1274
:10015000DB2A0830F80000008610831686100000A5
:100160008312B40D0610031CB828831606148312DC
:100170000318BD2883160610831283168614831273
:10018000861CC028F80BAB2800008610831686104A
:10019000000006140000000086148312861CCE287E
:1001A000F801000006187814861083168610831252
:1001B000061083160610831208000830B500770871
:1001C000B60083160614000086148312861CE628E7
:1001D00006180314061C0310F80D00008316861081
:1001E00083128610B50BE1288316061400008312D3
:1001F000061036080319FF28831606108312000024
:10020000831686148312861C032900008610831629
:1002100086100000831206108316061083128A11BE
:100220000A123C2B831603178C170C1400000000D5
:100230000318412983120C087F390313B6000317F2
:100240000D080313B70003170F080313B80036088F
:10025000BD003F20370803178D000313380803172C
:100260008F0083168C170C140000000083120313F8
:10027000B50B3B293E2983160317412960298316B4
:10028000031783120C0D0E0D7F390313B6000317ED
:100290000D080313B70003170F080313B80036083F
:1002A000BD003F20370803178D00031338080317DC
:1002B0008F008D0A03198F0A03100313B50B12293F
:1002C00008003C08F8013B02031869293B08F700C5
:1002D0007529F7010830BD00BB0DF70D3C0877020A
:1002E0000318F700F80DBD0B6C2908002030361EEE
:1002F0003030B7003508F700B51F8529F709F70A30
:100300007708B5002D30B700B6173508BB0064304C
:10031000BC0061217708B50030307807B800350897
:10032000BB000A30BC00612130307707BA003030A2
:100330007807B9003708F700B61DA029B61F361197
:10034000361AAD29B61FC8293619C8297708B8004A
:10035000B618C8297708B900C82930303802031DFB
:10036000C8297708B8002030B700B61DBB29361160
:10037000B614B61FB61030303902031DC8297708ED
:10038000B9002030B800B61DBB29B610B61F361014
:10039000361DCD293708BD003F20B61CD2293808AC
:1003A000BD003F20361CD7293908BD003F203A0840
:1003B000BD003F208A110A125F2BBC010408BB005C
:1003C0003C10831B3C14B51FED29BB173B1EBB0A19
:1003D000B409B509B40A0319B50A350EF038B700E7
:1003E000B707E23EB800323EBA0035080F39B80709
:1003F000B807BA07E93EB900B907B907340E0F3993
:10040000B907BA07B90DBA0DBA09BA0D34080F39D0
:10041000BA07B70D0730B6000A30BA07B903031C94
:100420000D2AB907B803031C112AB807B703031C28
:10043000152AB707B603031C192A36308400831324
:1004400007303B053B1384033B05031D2E2A3B1A53
:10045000840A3B1A2E2A2030F7004B2A84073A30B0
:10046000040203193B170008F700031D3F2A3B1B3A
:100470003F2A3B1A592ABB193F2A20304A2ABB1F60
:10048000472A2D30F70084033B13BB134B2ABB15BF
:100490003B123030F707B5010408B4003510831B58
:1004A00035147708BD003F203408840083133518C5
:1004B0008317840A3B1F2F2A0800353084008313DA
:1004C00000080319702A0230F800F701F70B662ABA
:1004D000F80B652A9730F700F70B6C2A800B632A1C
:1004E0008A110A12BF2B840183131F3083057130D8
:1004F00083168F000F088611831286158316031743
:100500000908C039890003131F129F120030031716
:1005100088008312870188018901FF300313A0003E
:10052000831603170908C039890003131F129F128D
:10053000003003178800831203131F139F138316C1
:100540009F1383121F149412A01220088316870091
:10055000831220162008831687008312A01120081A
:1005600083168700013083129400003083169400B4
:100570000108C73908388100831290010030F80063
:1005800092000030831692008312201520088316F3
:1005900087008312970183169B019C0101309D0007
:1005A0008312031787018801890104308D00003010
:1005B0008F0003136128A201A101A401A3018316E6
:1005C000061400008614000083120610831606101D
:1005D00000008312861083168610B4308312B40094
:1005E000A9207808331078183314831606100000F9
:1005F00086148312861CFA2A0000FE2A0000831645
:100600000614000001308312B306831606100000A2
:1006100086148312861C0A2B00000E2B0000831602
:100620000614000006140000861400008312061051
:100630008316061000008312861083168610B530CC
:100640008312B400A9200430B400A9208316061434
:100650000000861400008312861C2C2B06108316C3
:10066000061000008312861083168610B4308312A1
:10067000B400A920F701DD287808AE008316061023
:10068000000086148312861C432B0000472B0000B9
:100690008316061400000030831233180130B400B2
:1006A000103003178D0000308F0003100630031345
:1006B000B50012213408B5001F30B6007629143079
:1006C00003178D0000308F0003100D300313B500A9
:1006D00012211B3003178D0000308F0003100730EC
:1006E0000313B5001221103084002808B500270834
:1006F000B400DD21203003178D0000308F0003107F
:100700000C300313B5001221273003178D00003081
:100710008F00031007300313B5001221103084003E
:100720002A08B5002908B400DD212C3003178D00FC
:1007300000308F0003100C300313B500122133304A
:1007400003178D0000308F00031007300313B5002E
:100750001221103084002C08B5002B08B400DD21D4
:10076000383003178D0000308F0003100C30031356
:10077000B50012210830B400FA30B5005D2AB40B80
:06078000BC2BDB2A630024
:04400E00F52CFF3F4F
:00000001FF
